:100000008A010A285B2869287B288E289928AB2832
:10001000E228F22802208A110A1207208A110A1205
:100020003C308312AB0006208A110A120E30831274
:10003000AB0006208A110A1209208A110A12103018
:1000400083122502013003180301003C03194F28D5
:10005000A9080130031D0301003C03194E2801309B
:100060008312A9000A302502013003180301003C65
:1000700003194428A0012508303E0318A00AAA004D
:1000800004208A110A124E288312A0012508373E47
:100090000318A00AAA0004208A110A125428831205
:1000A000290803195428A90110308312A20008203E
:1000B0008A110A121C2883128501F83083168500E4
:1000C00006309F00831205100511851083168601E6
:1000D0000800FF30831686008312851483120511F1
:1000E000000005150000861B6E2805110000851014
:1000F0008316860108008312851005102A088600E1
:1001000003208A110A128312051405150000051137
:100110002D30A40005208A110A120800A40CA40C9A
:100120003F30A4050330A4020000A40B9428000073
:1001300008008312851005102B08860003208A1101
:100140000A1283120515000005112D30A4000520A8
:100150008A110A1208003C308312AB0006208A1173
:100160000A1205308312A20008208A110A123C30BC
:100170008312AB0006208A110A1205308312A200F6
:1001800008208A110A123C308312AB0006208A1123
:100190000A1205308312A20008208A110A120830C0
:1001A0008312AB0006208A110A1201308312AB00C1
:1001B00006208A110A1206308312AB0006208A112B
:1001C0000A1208008E308312A30000000000000015
:1001D000000000000000A30BE7280000A20BE228AB
:1001E00000000800F0308316860081138312860118
:1001F0000609A700A70EA601831227080139FF39B7
:100200000130031D0030003C03190B29270C7F39F6
:10021000A700A60AFC280430831226020130031826
:100220000301003C031948292608A8000F30831653
:1002300086008113831286010609A700A601831296
:1002400027080139FF390130031D0030003C031934
:100250002E29270C7F39A700A60A1F2904308312F4
:100260002602013003180301003C03194429260823
:10027000A700A0012808A100A10D210DFC39270726
:100280000318A00AA5004729FF308312A5004B29B7
:08029000FF308312A5000800F5
:00000001FF
